:100000006C28A301A200FF30A207031CA307031C56
:1000100067280330A100DF300F200328A101E83E4C
:10002000A000A109FC30031C1828A00703181528FC
:10003000A0076400A10F152820181E28A01C222844
:10004000000022280800A101A301A20002303028EC
:10005000A20003303028A20006303028A20005306C
:10006000A80023082102031D37282208200204309B
:1000700003180130031902302805031DFF306728DB
:100080000038031DFF300405031DFF3067280404FA
:10009000031DFF306728A501A4011030A600210D23
:1000A000A40DA50D2208A4022308031C230FA502FA
:1000B000031861282208A40723080318230FA507A3
:1000C0000310A00DA10DA60B4F282008672883134D
:1000D0000313831264000800FF2383169000831229
:1000E00083160510851405118511051285168312D6
:1000F0000730990083169F01811399019614961673
:100100008312C001C101C2014414C414BE01BF0165
:100110009130C300332205150000000000000000EC
:1001200000000000000005110000000000000000B9
:1001300000000000000000000000000000000000BF
:1001400000000000000000000000000000000000AF
:10015000C30B8B28080005150000000000000000FC
:100160000000000000000511000000000000000079
:10017000000000000000000000000000000000007F
:1001800000000000000000000000C30BAB280800C6
:100190000515000000000000000000000000000045
:1001A0000511000000000000000000000000000039
:1001B000000000000000000000000000000000003F
:1001C000C30BC8280800051500000000000000004F
:1001D0000000000000000511000000000000000009
:1001E000000000000000000000000000000000000F
:1001F00000000000C30BE328080005150000000004
:1002000000000000000000000000051100000000D8
:1002100000000000000000000000000000000000DE
:1002200000000000C30BFD280800051500000000B9
:1002300000000000000000000000051100000000A8
:10024000000000000000C30B152908000B108B15DF
:100250006300000000000B108B112E290030851A5E
:100260000130A00000302320B2000030C41801305B
:10027000A00001302320B40032088400340840205C
:10028000B400B50064003408350403194E2905167E
:10029000831605128312BE01BF01C41000308518F9
:1002A0000130A00000302320B2000030441801309B
:1002B000A00001302320B40032088400340840201C
:1002C000B400B5004208A00000302320B600340876
:1002D0003504840036084020B600B70064003608B4
:1002E0003704031994290516831605128312BE01DB
:1002F000BF017B304007B20002300318013E4107C6
:10030000B3003208A0003308A100FD30A300E8309C
:100310002820031D91297B30C00702300318013EBD
:10032000C1070130C20044108B200511831605114E
:10033000013083120120AB20051183160511013015
:1003400083120120C8200511831605110130831284
:100350000120E320051183160511013083120120CD
:10036000FD2005118316051101308312012015218E
:1003700005118316051183120330A10020300F20D0
:100380004008A0004108A100A30100302B20031D5C
:10039000CF290130C0020030031C013EC1026400BD
:1003A00001304202031CD529C2036400851CD929EF
:1003B00044146400851EDD29C4144008A0004108CF
:1003C000A100A30100302520B2000030851A0130C1
:1003D000A00001302320B4003208840034084020FB
:1003E000B400B5006400340835040319002A05126E
:1003F000831605128312051183160511831226290F
:10040000BE0A0319BF0A3E08A0003F08A100283019
:10041000A200A3014B202408B2002508B300320833
:10042000A0003308A100A30100302E20031D1D2AC7
:100430000516831605128312212A0512831605124A
:1004400083122E2905168316051283120130A3008C
:100450002C30022005128316051283120130A300EE
:100460002C30022008000511831605118312222268
:10047000222222220030851A0130A00000302320E1
:10048000B200003085180130A00000302320B400F5
:100490003208840034084720B400B50064003408F2
:0E04A00035040319542A2E2926296300552AF3
:02400E00D43F9D
:00000001FF
